:020000040000FA
:0600000000000DEF00F00E
:02000800FFD720
:08001800FFD70AD882748ED8CC
:10002000BAD8E2D892D80D060C0601E20B8AF6D7B0
:100030008E0EC16EE10E926ECC0E936EF00E946E2B
:100040000F0E956E000E966E880ED56E100E806E99
:1000500036D883CF05F0076A080E086E096A010ECC
:100060000A6E070EF76EC40EF66E47D8070EF76ECF
:10007000CE0EF66E42D8070EF76ED80EF66E3DD84D
:10008000070EF76EE20EF66E38D8070EF76EEC0E1E
:10009000F66E33D8070EF76E240EF66E2ED8140EB9
:1000A0000C6E81829E86200EC66E400EC76EA66ABA
:1000B000A188C00EF26E800ED06ED6DA12000A0E43
:1000C000026E43D80206FDE18490070EF76E1C0E07
:1000D000F66E08008482F5CF83FF849236D884823E
:1000E000F538836E849231D80B00F552F3E112009B
:1000F000210E026E0206FEE1120084900800F55205
:1001000001E10B008482F5CF83FF84928482F5386D
:10011000836E8492EDDF84800B00F552F3E11200D0
:1001200084908482EFCF83FF84928482EF38836E41
:100130008492DEDF8480EC50F4E1120080880406B3
:1001400003E1FA0E046E80981200F2A4FED7F29E2C
:10015000D6CF00F0D7CF01F0660E00269E0E01220A
:1001600001C0D7FF00C0D6FFF294F28E1200066ADB
:100170008350036E0518030B0BE0053002E3E89291
:1001800001D0E8820318030B02E1060601D0062A1B
:1001900003C005F012000890089283A602D00888D8
:1001A00001D0089808A604D008B802D01E0E096E27
:1001B00008B807D0095204E108B402D008800884C6
:1001C00001D0089408B607D008A805D0095201E06C
:1001D00008820894096A095201E0090608A802D0B9
:1001E000088601D00896120008A013D00A2A070E2C
:1001F0000A5C02E1010E0A6E070EF76EA60EF66E9D
:100200007CDF070EF76EB00EF66E77DF0B940B9661
:100210000B980A50010821E108A006D0070EF76EDE
:10022000240EF66E7DEC00F00B900B9208A207D026
:100230000B7CC00E0B14A86E010EA96E43DA0BAA3C
:100240000CD0D9D80BBC04D0200E1126E86A12229B
:1002500046DA93D90B9A140E0C6E0A50020812E17A
:1002600008A006D0070EF76E2E0EF66E7DEC00F09D
:1002700008A207D00B7EC00E0B14A86E010EA96E4B
:1002800021DA4FD90A5003080CE108A006D0070E66
:10029000F76E380EF66E7DEC00F008A201D00B7000
:1002A0004DD90A50040819E10BB00BD0010E0A6EAB
:1002B00008A006D0070EF76E240EF66E7DEC00F057
:1002C00009D008A006D0070EF76E380EF66E7DEC4A
:1002D00000F041D908A201D00B720A50050840E194
:1002E00008A006D0070EF76E380EF66E7DEC00F013
:1002F00008A006D0070EF76E840EF66E7DEC00F0B7
:1003000008A006D0070EF76E720EF66E7DEC00F0B8
:1003100008A223D00BB821D00B880B840F6A0FC022
:10032000A8FF020EA96ECED9640E106E10C0A8FFF1
:10033000030EA96EC7D90A0E0E6E640E0D6E070E5F
:10034000F76E780EF66ED9DE070EF76EF60EF66EC5
:10035000D4DEF7CF29F0F6CF2AF00BA801D04CD984
:100360000A50060847E10BB20BD0010E0A6E08A036
:1003700006D0070EF76E240EF66E7DEC00F03AD034
:1003800008A006D0070EF76E380EF66E7DEC00F072
:1003900008A006D0070EF76E8C0EF66E7DEC00F00E
:1003A00008A006D0070EF76E720EF66E7DEC00F018
:1003B00008A21DD00BB81BD00B880B86640E106EE4
:1003C00010C0A8FF030EA96E7DD90A0E0E6E640E32
:1003D0000D6E070EF76E780EF66E8FDE070EF76E57
:1003E000F60EF66E8ADEF7CF29F0F6CF2AF00BA8CC
:1003F00001D002D9120081929E96FF0EC96E9EA670
:10040000FED7C9CF12F09E9612C0C9FF9EA6FED796
:10041000C9CF11F0818211A807D0070EF76EBA0E6E
:10042000F66E6BDE0B9801D001D812000BBE03D024
:10043000050E1C6E02D0030E1C6E6DD812C02CF07F
:1004400011C02DF00BBE08D00BAC03D07D0E356E65
:1004500002D0E10E356E07D00BAC03D0190E356E0D
:1004600002D02D0E356EC5EC06F00BBE05D0030E86
:10047000356EE80E366E03D0356A640E366E0BECC0
:1004800006F02DC012F02EC011F00BAC02D00F50B0
:100490000BD00FC02CF0090E356EBEEC06F0050E29
:1004A000356E56EC05F02D50115EE86A125A02E2E4
:1004B000126A116A12C02CF011C02DF00BAC03D0DF
:1004C000640E356E02D0B40E356EC5EC06F02CC04D
:1004D00013F02DC012F02EC011F00BAC03D010C0E1
:1004E00035F00CD010C02CF0090E356EBEEC06F0C5
:1004F000050E356E56EC05F02DC035F013C02CF00E
:1005000012C02DF011C02EF097EC05F02DC012F0A6
:100510002EC011F01200D890123211321C06FBE1ED
:1005200012000BBE05D0070EF76E5E0EF66E04D0FD
:10053000070EF76E680EF66EE0DD12000BB005D008
:10054000070EF76E4A0EF66E04D0070EF76E540EC5
:10055000F66ED3DD12000BB205D0070EF76E9E0EBD
:10056000F66E04D0070EF76EA20EF66EC6DD070E0D
:10057000F76E940EF66EC1DD12000BBC05D0070EAF
:10058000F76E420EF66E04D0070EF76E460EF66E4C
:10059000B4DD12000BAA0DD00BBC05D00B8CFBEC0C
:1005A00001F00B9C02D0FBEC01F004D80B9A140E66
:1005B0000C6E120000EE24F010EE26F0EDCFE5FFF9
:1005C000E9281D08FBE112C0ECFF11C0ECFF12008E
:1005D00000EE26F0286A276AED502826ED502722E3
:1005E000E9281D08F9E127C02CF028C02DF0050EE0
:1005F000356E56EC05F012000D5234E10E0624E182
:100600000B98070EF76E7E0EF66E77DD0BA410D0FA
:100610000B94DEDF2D500F6E0FC0A8FF020EA96EE7
:1006200051D8640E106E10C0A8FF030EA96E4AD8F0
:100630000BA609D00B96CCDF2D50106E10C0A8FF72
:10064000030EA96E3FD80ED029C0F7FF2AC0F6FFCF
:10065000640E0D6EF62AE86AF7224FDDF7CF29F017
:10066000F6CF2AF097DF1200A96AA680A850AA0A3E
:1006700010E1010EA96EA680A8CF0BF0020EA96EA4
:10068000A680A8CF0FF0030EA96EA680A8CF10F009
:1006900018D0AA0EA86E000EA96E14D80B6A0BC053
:1006A000A8FF010EA96E0ED80F6A0FC0A8FF020E98
:1006B000A96E08D8640E106E10C0A8FF030EA96EB4
:1006C00001D81200A198A684F29E550EA76EAA0E1C
:1006D000A76EA682A1A8FED7A694F28E120000EE05
:1006E0001AF012C02CF011C02DF00A0E356E818068
:1006F00056EC05F0819030503009ED6E2C502D10E5
:10070000F6E1E950140805E0200EED6EE9501408FA
:10071000FBE1C00EEF6E1B6A03DD120033322801CD
:100720000C06000080202054454D502020008043BE
:100730004849502053454C008043414C4942524166
:100740005400C6DF4600C6DF4300C0202020202022
:10075000204E4F00C0202020202059455300C020AB
:100760002020203636373400C0202020203636376F
:100770003500C542474E0000C52020202000C54559
:100780004E44000000C04652455A200000C0424F6F
:10079000494C200000C120504F494E54200000C059
:1007A000310000C0320080202020202020202000A6
:1007B000C0202020202020202000C0204552524F61
:1007C000522020004880809090908080800050804F
:1007D00080989898808080005880809C9C9C808025
:1007E00080006080809E9E9E808080006880809FC8
:1007F0009F9F8080800000C6010000C6020000C6E6
:10080000030000C6040000C60500C6050100C605B9
:100810000200C6050300C6050400C6050500000069
:1008200001000180565501403433AB2A9324012046
:10083000721C9A1946175615B2134A12121101105A
:10084000100F390E7A0DCD0C310CA30B220BAB0A15
:100850003E0AD9097C092509D408890843080108FA
:10086000C207880751071D07EC06BD0691066706FB
:100870003F061906F505D205B10591057305560524
:100880003A051F050605ED04D504BE04A80493042B
:100890007E046A045704450433042204110401044D
:1008A000F103E103D303C403B603A9039C038F033D
:1008B000820376036A035F03540349033E03340350
:1008C0002A03200316030D030403FB02F202E902CC
:1008D000E102D902D102C902C102BA02B202AB02DC
:1008E000A4029D0296029002890283027D02770291
:1008F00071026B0265025F025A0254024F024A0201
:1009000044023F023A02350231022C02270223023E
:100910001E021A02150211020D020902050201024D
:10092000FD01F901F501F101ED01EA01E601E20144
:10093000DF01DB01D801D501D101CE01CB01C80116
:10094000C401C101BE01BB01B801B501B301B001D1
:10095000AD01AA01A701A501A2019F019D019A0174
:1009600098019501930190018E018B018901870106
:100970008401820180017E017B017901770175018B
:10098000730171016F016D016B01690167016501FF
:10099000630161015F015D015B015901580156016D
:1009A0005401520151014F014D014B014A014801CF
:1009B000470145014301420140013F013D013C0126
:1009C0003A01390137013601340133013101300177
:1009D0002F012D012C012A012901280126012501C1
:1009E00024012201210120011F011D011C011B0105
:1009F0001A01190117011601150114011301120141
:100A000010010F010E010D010C010B010A0109017A
:100A100008010701060105010401030102010101AA
:100A2000100E356008D035B6100C35B4200C35B238
:100A3000400C35B0800C35BC020C35BA040C35B80E
:100A4000080C2FC033F02F6A2EC032F02E6A2DC052
:100A500031F02D6A2CC030F02C6A000C306A000C8A
:100A6000010E35642EEF05F02CC030F035502C60AF
:100A700002D02C6A000CD890F76AE836F7361F0FC0
:100A8000F66E080EF7220A00F5503002F4CF2CF073
:100A9000F3CF2DF00800F5503002F4502D26E86A0F
:100AA0002C2235502C02F350305E000C010E3564C0
:100AB0002EEF05F0D890F76A3534F7361F0FF66E33
:100AC000080EF7220A002CC031F02DC030F0F5508E
:100AD0003102F4CF2CF0F3CF2DF00900F5503002A5
:100AE000F4CF2EF03102F3502E26F4502D22E86A76
:100AF0002C220A00F5503002F3502E26F4502D22FD
:100B0000E86A2C2235502D02F3CF2FF0F4CF2EF0CF
:100B10002C02F3502E262F50305E2E50315A31AE1B
:100B2000000C2D06E86A2C5A35503026000C2CC0DB
:100B300042F02DC043F02EC044F056EC05F02CC01E
:100B400042F02DC043F044C02DF030C02CF056ECE4
:100B500005F02DC02EF043C02DF042C02CF0000C4B
:100B6000356608D036C035F056EC05F030C031F0AF
:100B7000306A000C35502C5CD8A027EF05F0D8A4C3
:100B800005D036502D5CD8A027EF05F02CC042F0E0
:100B90002DC043F02DC03CF02CC02DF02C6A35C088
:100BA00037F036C038F035BE1DD03550E846210F3D
:100BB000F66E080EF76AF7220800F5503802F3CFF8
:100BC00036F0F4CF35F03702F3503526F5504302B6
:100BD000F3CF3CF0F4CF2DF04202F3502D262C6AD7
:100BE000F4502C225AEC05F02D503602F3503C5CA8
:100BF000F4503058D8A02D062D503802F350435EE3
:100C0000F450425A2D503702F350425E42C030F049
:100C100043C031F0000C306A316AE86A356608D0AA
:100C200036C035F097EC05F030C031F0306A000C7A
:100C30002C620CD02DC02CF02EC02DF0B0EC05F0A5
:100C40002DC02EF02CC02DF02C6A000C2EC02FF0E1
:100C50002DC02EF02CC02DF02C6A2CC042F02DC0DF
:100C600043F02EC044F02FC045F0020E2B6E010E53
:100C70003E6E35BE1CD010EC05F03E6E360235508F
:100C8000F3CF36F0F4CF35F03E02F35035263E5028
:100C90002F02F3CF45F0F4CF44F02D02F3CF43F011
:100CA000F4CF42F02E02F3504426F4504326D8905D
:100CB000F76A3534F7361F0FF66E080EF7220A0072
:100CC00042C02CF043C02DF063EC05F02CA008D0FE
:100CD0002D6843C030F035503026D8B085EF06F08F
:100CE0002D503602F350445CF4503058D8B00DD03B
:100CF0002D0635503026D8B008D02D503602F3508E
:100D0000445CF4503058D8A02D062DC03FF02D5033
:100D10003602F350445EF450435A2D503502F350DE
:100D2000435EF450425A42AE05D03F063650442648
:100D3000355043222B4E09D03FC040F043C042F013
:100D400044C043F045C044F0BBD743C030F044C07A
:100D500031F0010E3E640CD03E40356E10EC05F0D3
:100D60004402F4CF31F04302F3503126F4CF30F097
:100D70002C6A3FC02EF040C02DF0000C35502C02E4
:100D8000F4CF2CF0F3CF2DF0000C35502D02F4CF22
:100D90002DF0F3CF2EF02C02F4CF2CF0F3502D26B3
:060DA000E86A2C22000CA1
:020000040030CA
:08000000FFFAFCFEFFFF01FF07
:00000001FF
